:0200000057287F
:08000800562882070834003479
:1000100098349634803486348634073400340F3470
:100020004234403487348734063400340134863413
:10003000A034C034C03405340034003427341034C4
:10004000C234C1340434003400340334E834C334DB
:10005000C33403340034003400346434C434C4344E
:1000600002340034003400340A34C634C534013458
:100070000034003400340134C734C734FF348207FD
:100080000134563446344F342B3449344634023428
:10009000493446342D34563446344F3403345634C0
:1000A00046344F342D3449344634FF340900850139
:1000B00086018316FF3085000030860027308100DE
:1000C0008312FB223F2396228101B7010B11051DEC
:1000D00074288316FF30850083123F238511831611
:1000E000F730850083127E288316FF308500831247
:1000F000462385118316F73085008312AF20C32075
:10010000051C8428332364283F23051C84280730DA
:10011000BB00D0221121DA22051C9628851C9128CB
:100120008C283F23851C912823218A283F23051CE6
:100130009628BB0B8A28D5221F21051CAA28851CBE
:10014000A2289D283F23851CA228B00BA928033094
:10015000B0009C283F23051CAA280A236428010814
:10016000B8000B1DB528B70A0B11BA01BA038511E7
:100170008515010838020319BE28C028BA0AB72815
:100180003A09B90008003008B00BD428B0008E013D
:1001900037088F0038089000390891000E30B200FF
:1001A0002C30B1008B210429B00BF128B000920152
:1001B0003708930038089400390895002C30B100B6
:1001C0000E30B20004308D00D7210E30B200123054
:1001D000B100AD21160B04298E018F019001910110
:1001E0000429B0008E0137088F00380890003908C4
:1001F00091000E30B2002C30B100AD21160B042955
:100200008E018F01900191010E30B1002830B200B3
:1002100004308D00D721E421BE0100226722B722DD
:1002200008002C30B1002830B20004308D00D721F6
:10023000E4210130BE0000227422B72208006321AD
:100240008122B72208002C30B1002830B2000430DF
:100250008D00D721E4213B08083C203E8400800A21
:100260000A3000020319800148222C30B2002830E5
:10027000B10004308D00D72108000301B40005202F
:10028000B600FF303602031962293608330203191B
:100290004C293408073E3E293408013E05209200CF
:1002A0003408023E052093003408033E05209400E4
:1002B0003408043E052095003408053E051D013E26
:1002C0000520960008000301B4003F20B600FF306F
:1002D000360203198A2936083002031972293408B4
:1002E000073E64293408013E3F20A2003408023E44
:1002F0003F20A3003408033E3F20A4003408043EFE
:100300003F20A5003408053E3F20A6003408063EE5
:100310003F20A7000800960104308D000330B1078C
:100320000330B20732088400160880079601031CC8
:100330009B2901309600310884000008B40032087F
:10034000840034088007031CA729013096008D0B18
:10035000AA290800B103B2039229960104308D0046
:100360000330B1070330B207320884001608800258
:1003700096010318BD290130960031088400000859
:10038000B40032088400340880020318C9290130FF
:1003900096008D0BCC290800B103B203B429970154
:1003A000AD21970A160BD0298B219703080031083D
:1003B00084000008B4003208840034088000B10AC8
:1003C000B20A8D0BD729080028088E0029088F0053
:1003D0002A0890002B0891000830B30020308400D8
:1003E0000E30B2001230B1000408B5003D21CF211B
:1003F0003508840017088000840AB30BF42908002C
:10040000051D102A2030B1001E30B20003308D00CF
:10041000D7212330B1002230B20003308D001D2AD5
:100420002030B1001E30B20004308D00D7212430BE
:10043000B1002330B20003308D00D7212022080004
:100440000A308D001E3084000730051D06300D0275
:100450000319302A0330051D02300D02031D352A11
:100460002030BE08031D2E30422A00080319392A05
:10047000402ABE08031D3E2A203E422A303E422A20
:10048000BE0A303E80008D0B462A0800840A242ACA
:10049000A801A901AA01AB010830B30020308400F3
:1004A0002830B2001230B1000408B5003D213508F3
:1004B00084000008BC00BC080319612A8B21BC031E
:1004C0005B2A35088400840AB30B542A080046309E
:1004D00098007230990065309A0071309B002E3080
:1004E0009C003A309D000800493098004630990041
:1004F00073309A0065309B0074309C003A309D0048
:1005000008004D3098006F30990064309A006530D3
:100510009B0020309C0073309D0065309E0074303D
:100520009F003A30A0002030A10008002330860050
:1005300086123F232330860086123F232330860015
:1005400086123F232230860086123F2328308C00FB
:10055000E1223F2306308C00E1223F230C308C0047
:10056000E1223F2301308C00E1223F23080080304C
:100570008C00E12208308D001830840000088C00C7
:10058000EE22840A8D0BBE2AC0308C00E122083096
:100590008D0000088C00EE22840A8D0BC92A080009
:1005A0000D308C00E1223F2308000C308C00E1224A
:1005B0003F2308003B08B3003D2116088C00E122D0
:1005C00008000C0E0F3920388600861250230C08C4
:1005D0000F39203886008612502308000C0E0F3980
:1005E00030388600861250230C080F3930388600C8
:1005F00086125023080005308D0089012C308400BC
:1006000083160814831208088000890A840A8D0B57
:10061000002B080005308D0089012C3084008316E2
:100620000815831200088800831655308900AA3007
:1006300089008814081E1A2B08128312890A840A5A
:100640008D0B122B83120800C530BA00272BBA0B72
:10065000262B0B1D2E2BB70A0B11302B0000302B35
:100660000000322B080024232423242324232423C2
:10067000242324232423242324233E2B08000A306C
:10068000BD003323BD0B412B452B08002030BD009E
:100690003323BD0B482B0930BD00BD0B4D2B08008B
:0E06A0001430BD0000000000BD0B522B0800FE
:02400E00F93F78
:0A42000000000000000000000100B3
:00000001FF
